:020000040000FA
:10000000640085010730242829298A018207122BE0
:100010001D2B282B332B3E2B492B542B5F2B6A2B6C
:10002000752BB100093C0318172803011828310863
:100030008A018207922B972B9C2BA12BA62BAB2BF3
:10004000B02BB52BBA2BBF2B9F008601023090003E
:100050008F018E010C10831613309200073081003F
:10006000003085007730860001308C00831202302A
:100070009500043092000C309700203084008001FD
:10008000840A0408803A031D3F2828258517FF2489
:100090002130FC240C3060258038FC240630FC2400
:1000A0001330FC242030FC240C30FC2403011425E4
:1000B0002025DB2420308400831600309B001C1494
:1000C0001A088000840A9B0A1B080C3A031D5F284B
:1000D0008312FC2152247124FF30AF008101F030E3
:1000E0008B002C1F7C28061DD60110305602031CE5
:1000F0007C282C13AC12D6016400AC1952242C1AA3
:100100007124AC188424061A382D2C1F90282C1C1E
:100110007128B701B801B901FC21BA012C1071286E
:10012000AC1EA1280619A42820305602031C8728DB
:10013000A701A601A501AB01AA012C162C17D60117
:100140008728061DAC16872802305602031C0F298B
:100150001325D6012025F7210F30E0210A30E021B8
:100160000C30E0211B2148088023232112218030FC
:10017000B5004130B6002425F7210A30E0210B30CC
:10018000E0210C30E0211B214B08BD004C08BB00D6
:10019000BC01BF015408BE005508C000A22443089A
:1001A0008023232112218030B5004330B60024255E
:1001B000F7210D30E0210C30E0210E30E0211B2131
:1001C0004F08E0214E08E0214D08E021F7211130D1
:1001D000E0211230E0218030B5004530B600242502
:1001E000F7210E30E0211030E0210E30E0211B21FC
:1001F0005308802325211E215108802325211E21FB
:1002000052088023252156082D3A031DAA28AC1236
:10021000061DAA281325AC152C163A089F24AC12EB
:10022000D6018728F7211130E0211230E021133068
:10023000E0211430E029F721F721F7293630F9249D
:100240003630F924F82C3908E0213808E021370845
:10025000E0296400F0000308F10083010B19C329B1
:100260000C18BA291014AF0A2F08063A031D4329A7
:10027000AF0110100F08AD000E08AE008F018E0107
:1002800010140C1CAC14A80A0319A90A2908173A5F
:10029000031D6F292808703A031D6F29AC15A801AA
:1002A000A901A40A0A302402031C6F29A401A30A8D
:1002B0000A302302031C6F29A301A20A0A3022027A
:1002C000031C6F29A201A10A0A302102031C6F2915
:1002D000A101A00A0A302002031C6F29A001AA0A6A
:1002E0000319AB0A2B08173A031D8F292A08703A05
:1002F000031D8F292C16AA01AB01A70A0A30270279
:10030000031C8F29A701A60A0A302602031C8F2985
:10031000A601A50A0A302502031C8F29A501C90AD6
:100320000319CA0A4A08173A031DB4294908703A42
:10033000031DB429C901CA013C30CB070318CC0AFC
:10034000CD0A0A304D02031CB429CD01CE0A0A3071
:100350004E02031CB429CE01CF0A0A304F02031CFF
:10036000B429CF01CB01CC018B1071088300F00EB2
:10037000700E09002C14AC1010108F018E01FF308C
:10038000AF000C10B529AC1AD60A0B11D00A5008D0
:10039000103A031DB529D001D20A521CD00A5208C6
:1003A0003C3A031DB529D201D20AD50A0319D40A51
:1003B000D10A51083C3A031DB529D30AD101B52908
:1003C000B300B30A0830B2000530B1003108B207FB
:1003D000B30BE62932086025F924B20AB10BEA29E9
:1003E000F82CF8246030F9246030F924F82CF82433
:1003F000F824F824F824F82C6400A630B500403026
:10040000B6002425DD22E122F824B60A2425DD22C7
:10041000E122F824B60A2425DD22E122F824B60AD6
:100420002425DD22E122F8243908031D1B2A38087F
:10043000031D2A2A302AA630B5004030B6002425F4
:100440004022B60A24254522B60A24255322B60A9C
:100450002425C522AD30B5004030B600380805204F
:10046000C230B5004030B600370805281023EC2212
:10047000EE22F022E122F022EE22EC22102BDD22ED
:100480000023F022EE22EC2ADD22F222F422F622D0
:10049000102B1023F622F422F222E122F222F4227F
:1004A000F622102BDD22F022EE22EC22102BEC2281
:1004B000F822FA22FC220F30E222FC22FA22F82251
:1004C000EC2A1023F6220223FE22C030E222FE2272
:1004D0000223F622102B1023EC22F822FA220330FA
:1004E000E222FA22F822EC22102BF6220223FE222C
:1004F0000423F030E2220423FE220223F62AF82409
:10050000062308230A230F30E222FC22FA22F822D3
:10051000EC2AF824F8240C230E23C030E222FE2219
:100520000223F622102B1023EC22F822FA220823B1
:100530000330E2220623F824F82CF6220223FE22BE
:100540000423F030E222EA220E230C23F82CF824B4
:10055000F824062308230330E222FA22F822EC22B0
:10056000102BF8240C230E23EA22F030E22204237D
:10057000FE220223F62AEC22EE22F0220023E122C0
:100580000023F022EE22EC2ADD22F222F422F622CF
:10059000102BEC22F822FA22FC220F30E2220A234E
:1005A00008230623F82C1023F6220223FE22C03053
:1005B000E2220E230C23F824F82CF824F824F82443
:1005C000F8240301B2000A30B1003208F924B10B5B
:1005D000E52A0800E030F92CFE30F92CFC30F92C2B
:1005E000F830F92C1F30F92C3F30F92C7F30F92CE2
:1005F000FD30F92CFB30F92CF730F92CDF30F92CD9
:10060000F030F92CBF30F92CEF30F92C0130F92CF7
:100610000330F92C0730F92C8030F92CC030F92C3C
:10062000FF30F92C24255722B60A24254922B60A80
:1006300024253622B60A2425752A24253F22B60A07
:1006400024254422B60A24255222B60A2425C42A87
:1006500024257F22B60A24258922B60A242593223E
:10066000B60A24259D2A24257F22B60A242589221C
:10067000B60A2425A722B60A2425B12A2425BB229E
:10068000B60A24256122B60A2425A722B60A242503
:10069000C42A2425C922B60A2425D322B60A242531
:1006A000A722B60A2425B12A2425C922B60A242560
:1006B000D322B60A24256B22B60A2425752A2425BE
:1006C0005722B60A24254922B60A24255222B60A00
:1006D0002425C42A24255722B60A24256122B60AD5
:1006E00024256B22B60A2425752A24255722B60A0A
:1006F00024256122B60A2425A722B60A2425B12A78
:10070000B700B801B9010A303702031C8A2BB700C1
:10071000B80A832B0A303802031C912BB800B90A9F
:100720008A2B080024253724B60A24252C2C2425BE
:10073000C423B60A2425D02B24250124B60A242557
:10074000112C24250124B60A24251F2C2425E82356
:10075000B60A2425F42B2425D823B60A24251F2CD9
:100760002425D823B60A2425472C24253724B60A65
:100770002425D02B24253724B60A2425472C2425CC
:100780003724B60A24251F2CF824F824F824F8244A
:100790003030F9243030F924FC30F924FC30F92CC5
:1007A000F824F824F824F824F824F8241023102B33
:1007B000FC30F924FC30F9240C30F9240C30F924F5
:1007C0000C30F9240C30F9240C30F9240C30F92CBD
:1007D000FC30F924FC30F924F824F824F824F82417
:1007E000FC30F924FC30F92C0330F9240330F924CF
:1007F0000330F9240330F9240330F9240330F924B9
:10080000D62B0C30F9240C30F9240C30F9240C30A0
:10081000F9240C30F9240C30F924FC30F924FC3094
:10082000F92C10231023C330F924C330F924C3302A
:10083000F924C330F924C330F924C330F92CC33070
:10084000F924C330F924C330F924C330F924C33068
:10085000F924C330F924D62B10231023C030F924F7
:10086000C030F924C030F924C030F924D62BFC3034
:10087000F924FC30F9240C30F9240C30F9240C3024
:10088000F9240C30F924FC30F924FC30F92C102325
:100890001023C330F924C330F924C330F924C33002
:1008A000F924D62BAC11CC30B5004430B600240866
:1008B0001120C230B5004430B60023081120B830F2
:1008C000B5004430B60022081120AE30B5004430E7
:1008D000B60021081120A430B5004430B60020082D
:1008E00011282C128030B5004430B60025081120A4
:1008F0008A30B5004430B600260811209430B50087
:100900004430B600270811280230BC00BF30BB00BD
:100910002030BD00BF018B132D08BE002E08C00083
:100920008B17A224430848020318982C4308C800D8
:10093000AC1043083A06031908004308BA008023A4
:10094000FC21080064003E08031DAB2C4008031D79
:10095000AB2CC30108001830C700C201C101C3019C
:10096000C501C401C6010310BD0DBB0DBC0DC60DF4
:10097000C40DC50D3F084502031DC42C3E084402AA
:10098000031DC42C40084602031CD52C4008C60297
:10099000031CC4034408FF3A0319C5033E08C402FC
:1009A000031CC5033F08C5020314C30DC10DC20DCE
:1009B000C70BB32C0800F721F721F7210A30E021FB
:1009C0001530E0211030E021F7210B30E02102301A
:1009D000E021F1210030E0210230E0211230E0215D
:1009E0002825282528256400061AF32C0301142D38
:1009F0000301B0008517032DB0008513032D0513E7
:100A000028250517003405110830B4008510B01BE7
:100A10000514B01F0510640085140000B00DB40B60
:100A2000062D051500340301B3000830B200FF3075
:100A3000B1003308F924B10B192DB20B172D0800A2
:100A40008030B5004030B6003508FC243608FC2C58
:100A500064000730B30064003230B1006400FA3043
:100A6000B200B20B312DB10B2E2DB30B2B2D003458
:100A70008B1320308400B101310860250006031D6E
:100A80005225840AB10A31080C3A031D3C2D132566
:100A90008030B5004530B6002425DB246400061AFA
:100AA0004E2D0028000883169A001C1555309D0015
:100AB000AA309D009C1464009C185B2D83120800D2
:0E0AC000640083169B001C141A0883120800A1
:02400E00143F5D
:10420000010002000500030002000600060006008F
:1042100000000000000000003F003E005100490087
:1042200045003E00000042007F00400000004200C8
:1042300061005100490046002100410045004B004B
:1042400031001800140012007F0010002700450004
:104250004500450039003C004A0049004900300053
:104260000100710009000500030036004900490003
:104270004900360006004900490029001E007E0062
:104280001100110011007E001F00200040002000DE
:104290001F00460049004900490031007F004100ED
:1042A000410022001C00010001007F00010001000C
:1042B0007F0002000C0002007F007F00090019004F
:1042C000290046007F0008001400220041007C0005
:1042D000040018000400780020001000080004000A
:1042E00002007F0008000400040078003E00410046
:1042F000490049007A0055002A0055002A0055005F
:00000001FF
